:04000000020A2E3290
:01000B0032C2
:0100130032BA
:01001B0032B2
:0100230032AA
:01002B0032A2
:100A2E007581071209A2E5826003020033020033CA
:1000330012085A80FE7A827B001ABAFF011BEA4B30
:1000430070F722AA82AB837C007D00C3EC9AED6437
:10005300808BF063F08095F0501AC002C003C00497
:10006300C005120038D005D004D003D0020CBC0068
:10007300DA0D80D7227A02DAFE227A00C3EA64809C
:100083009494500AC002120078D0020A80EE22C271
:10009300A712007DD2A712007D223098FDC2988559
:1000A30099821200B5859982223098FDC29885996C
:1000B3008222AA823099FDC2998A9922AA82AB83AD
:1000C300ACF07D008D060DEE2AF582E43BF5838CC2
:1000D300F0120A06FE8E07BE000280178F82C0024E
:1000E300C003C004C0051200B5D005D004D003D0AE
:1000F3000280D1227ADD7B087C028A828B838CF09A
:100103001200BF22AA37BA0D127AA57B087C028A95
:10011300828B838CF01200BF1200F7227A007B00DF
:100123008A04BC0A02802E758211C002C003120029
:10013300B5D003D002C002C00312009DAC82D0032D
:10014300D0028C028A04BC0D027A0AEB2442A8E096
:10015300A6020B80CB1BEB2442A8E076007A007B3F
:10016300007C00EC2442F88605BD00028037E4F5EC
:100173004F754E0A8A828B83C002C003C004C00538
:10018300120983AE82AF83D005D004D003D002ED31
:100193003395E0F8ED2EFEE83FFFEE24D0FAEF347E
:1001A300FFFB0C80BE8A828B832230980912009D4C
:1001B300AA828A3780037537FF227AE27B087C02A2
:1001C3008A828B838CF01200BF1200F722AA82C3AB
:1001D30074099A400F74302AFB8B82C0021200B557
:1001E300D002800974372AFA8A821200B522AA82C1
:1001F30074F05AFBC4540FFB8B82C002C00312017C
:10020300D0D003D002740F5AFB8B821201D022AAE2
:1002130082AB838B047D008C82C002C0031201F188
:10022300D003D0028A821201F122AA82AB83754ED7
:1002330010754F278A828B83C002C003120944AC16
:1002430082AD83D003D00274302CFCE43DFD8C4896
:10025300754E10754F278A828B831209A6AA82AB2B
:1002630083754EE8754F038A828B83C002C00312E5
:100273000944AC82AD83D003D00274302CFCE43D3E
:10028300FD8C49754EE8754F038A828B83C002C08B
:10029300031209A6AC82AD83D003D0028C028D0376
:1002A300E4F54F754E648A828B83C002C003120942
:1002B30044AC82AD83D003D00274302CFCE43DFD0A
:1002C3008C4AE4F54F754E648A828B83C002C00367
:1002D3001209A6AC82AD83D003D0028C028D03E455
:1002E300F54F754E0A8A828B83C002C003120944FC
:1002F300AC82AD83D003D00274302CFCE43DFD8C82
:100303004BE4F54F754E0A8A828B83C002C00312F9
:1003130009A6AC82AD83D003D0028C028D03E4F531
:100323004F754E0A8A828B83C002C0031209A6ACA2
:1003330082AD83D003D00274302CFCE43DFD8C4CA1
:100343007C007D00EC2448F88606BE3010C3EC9494
:1003530005ED940050070CBC00EA0D80E78C028D7C
:1003630003BC050BBD0008EC24FFFAED34FFFB8A48
:10037300048B050ABA00010BEC2448F88682C002FC
:10038300C0031200B5D003D002C3EA9405EB940076
:1003930040DD223098091200ACAA828A37800375A7
:1003A30037FF22120396AA82AB83BA1310BB000D48
:1003B300120396AA82AB83BA11F6BB00F3227580AF
:1003C30020120078C2B4C2B4D2B4C2B39000641293
:1003D30000467580D0C2A79000C8120046D2A7D2AB
:1003E300B390006412004622E4F531F530C3E530E2
:1003F3009400E531648094A0502C758040120078FD
:10040300C2B4D2B4853038853139853890AA397B66
:10041300004302808AA07580001200920530E4B583
:100423003002053180C722E537B46532D2B3D2B486
:10043300D2B5D2B6D2B71200781203C1E4F531F5C2
:1004430030C3E5309405E53164809480500D120388
:10045300C10530E4B530EA053180E61201BD22E57D
:1004630037B4770280030204F6D2B3D2B4D2B5D242
:10047300B6D2B7D2A7120078E536B4FF02C2B39062
:100483000064120046E4F53BF53AE4F531F530AA91
:1004930030AB31C3EA953CEB953D504C758211125C
:1004A30000B5758040120078C2B4C2B4D2B48530AE
:1004B30038853139853890AA397B004302808AA078
:1004C3001200ACAA828A807582131200B5AA807BBF
:1004D30000EA253AF53AEB353BF53B12009205303D
:1004E300E4B53002053180A7D2B390006412004610
:1004F3001201BD22E537B47202800302058DE4F5D3
:100503003BF53AD2B3D2A7D2B4D2B5D2B6D2B775ED
:1005130034317A007B00C3EA953CEB953D400302FE
:10052300058A758000C002C003120078D003D00290
:10053300C2B4C2B4D2B48A388B39853890AC397D11
:10054300004304808CA0C2B5C002C003120078D05F
:1005530003D0027580FFAC807D00EC253AF53AEDBF
:10056300353BF53B858082C002C0031201F1D00305
:10057300D002D2B5C002C0031203A6D003D0020A30
:10058300BA00010B0205191201BD22E580B4FF0276
:10059300800B7534300540E4B54002054122E53750
:1005A300B46C028003020611D2B3D2A7D2B7D2B67B
:1005B300D2B5D2B47A60E4F531F530C3E5309403B3
:1005C300E5316480948050438A80C002120078D061
:1005D30002C2B4C2B4D2B4C2B3900064C002120067
:1005E30046D0027580D0C2A7C00212007DD002D2CD
:1005F300A7D2B3900064C002120046D00274102A3E
:10060300FA0530E4B53002053180B01201BD22E5B0
:1006130037B463267AE87B087C028A828B838CF06A
:100623001200BFE53AF4FAE53BF4FB74012AF582C4
:10063300E43BF5831202121201BD22D2A7D2B3C248
:10064300B4C2B5C2B7C2B6E4F53975383175903165
:100653007A007B004302808AA0C2B51200787580BD
:10066300FF858035C2B50538E4B5380205398538CC
:1006730090AA397B004302808AA0C2B51200787524
:1006830080FF8580362212063EE535B45102802A6A
:10069300E535B452028033E535B45502803CE53587
:1006A300B46102801DE535B462028026E535B46588
:1006B30002802FE535B4FF378030753E00753F105B
:1006C300802D753E00753F108025753E00753F20D7
:1006D300801D753E00753F208015753E00753F50A7
:1006E300800D753E00753F508005E4F53FF53EE40F
:1006F300F53BF53AE4F541F540D2A7D2B3C2B4D203
:10070300B7D2B6D2B57534317A007B00C3EA953ED1
:10071300EB953F5057758000C002C003120078D09C
:1007230003D002C2B4C2B4D2B48A388B39853890AC
:10073300AC397D004304808CA0C2B5C002C0031253
:100743000078D003D0027580FFAC807D00EC253AA1
:10075300F53AED353BF53BC002C00312058ED003DD
:10076300D002D2B50ABA00010B02070F22E537B453
:10077300730E12011FAA82AB838A3C8B3D1201BD0B
:1007830022E537B467028003020829120689E5359A
:10079300B4FF030208177AF57B087C028A828B83F5
:1007A3008CF01200BF8535821201F1E536B4FF0FDC
:1007B3007A027B097C028A828B838CF01200BFE56C
:1007C30036B4050F7A077B097C028A828B838CF00F
:1007D3001200BF7A0B7B097C028A828B838CF01216
:1007E30000BF85408285418312022D7A187B097CE4
:1007F300028A828B838CF01200BF7A1F7B097C02F2
:100803008A828B838CF01200BF853C82853D8312E4
:10081300022D800F7A317B097C028A828B838CF0D4
:100823001200BF1201BD22E537B4702A1206898572
:1008330035821201F175822C1200B5854082854103
:100843008312022D75822C1200B5853C82853D836F
:1008530012022D1201BD22E4F531F530E4F53DF528
:100863003C759852758920758DFDD28E12009D7A44
:10087300A57B087C028A828B838CF01200BF120056
:10088300F71201AD12010712077012042A12046253
:100893001204F71205A112061212078412082A8005
:1008A300E0220A0D20456173792D446F776E6C6FDA
:1008B300616465722056322E3020666F7220494380
:1008C300533839433532283531292028736463631B
:1008D3002076657273696F6E29000A0D203E000A47
:1008E3000D206F6B000A0D2043484B53554D203D9F
:1008F30020000A0D20666F756E6420383943002D81
:10090300313256002D3556000A0D206E6F6E626C23
:10091300616E6B2000206279746573000A0D20629A
:100923007974657320636F756E74657220000A0DA8
:10093300204E6F7420666F756E6420383943787863
:1009430000AA82AB837C007D007E10EB235401FF61
:10095300EBCA25E0CA33FBEDCC25E0CC33FDEF60D9
:1009630003430401C3EC954EED954F400CC3EC9546
:100973004EFCED954FFD430201DED08A828B83222C
:10098300AA83AB828BF0E54EA4F8A9F08AF0E54E7A
:10099300A429F98BF0E54FA429F5838882222275D7
:1009A300820022AA82AB837C007D00E54F235401A1
:1009B300FE7028AE4EE54FCE25E0CE33FF8E4E8F30
:1009C3004FC3EA9EEB9F500E8E4EEFC313C54E13DB
:1009D300C54EF54F80050D8D0480D0C3EA954EEBCF
:1009E300954F4009C3EA954EFAEB954FFBE54FC38C
:1009F30013C54E13C54EF54F8C051CED70DD8A8271
:100A03008B8322C8C0E0E5F0600D14600F14600F03
:100A130014601074FF800FA882E6800AE08007E468
:0B0A2300938003A882E2F8D0E0C82214
:00000001FF
